 cmapdump

 Timestamp is 4a8b38ec (Wed Aug 19 07:27:40 2009)

 Preferred load address is 00400000

 Start         Length     Name                   Class
 0001:00000000 0000d508H .text                   CODE
 0002:00000000 00000124H .idata$5                DATA
 0002:00000124 00000004H .CRT$XCA                DATA
 0002:00000128 00000004H .CRT$XCZ                DATA
 0002:0000012c 00000004H .CRT$XIA                DATA
 0002:00000130 00000014H .CRT$XIC                DATA
 0002:00000144 00000004H .CRT$XIY                DATA
 0002:00000148 00000004H .CRT$XIZ                DATA
 0002:0000014c 00000004H .CRT$XPA                DATA
 0002:00000150 00000004H .CRT$XPX                DATA
 0002:00000154 00000004H .CRT$XPXA               DATA
 0002:00000158 00000004H .CRT$XPZ                DATA
 0002:0000015c 00000004H .CRT$XTA                DATA
 0002:00000160 00000004H .CRT$XTZ                DATA
 0002:00000170 000015d8H .rdata                  DATA
 0002:00001748 0000004eH .rdata$debug            DATA
 0002:000017a0 0000000cH .rdata$sxdata           DATA
 0002:000017ac 00000004H .rtc$IAA                DATA
 0002:000017b0 00000004H .rtc$IZZ                DATA
 0002:000017b4 00000004H .rtc$TAA                DATA
 0002:000017b8 00000004H .rtc$TZZ                DATA
 0002:000017c0 00000494H .xdata$x                DATA
 0002:00001c54 00000014H .idata$2                DATA
 0002:00001c68 00000014H .idata$3                DATA
 0002:00001c7c 00000124H .idata$4                DATA
 0002:00001da0 00000518H .idata$6                DATA
 0002:000022b8 00000000H .edata                  DATA
 0003:00000000 00003c9aH .data                   DATA
 0003:00003ca0 00001c04H .bss                    DATA

  Address         Publics by Value              Rva+Base       Lib:Object

 0000:00000000       __except_list              00000000     <absolute>
 0000:00000003       ___safe_se_handler_count   00000003     <absolute>
 0000:00000000       ___ImageBase               00400000     <linker-defined>
 0001:00000000       _fz_throwimp               00401000 f   base_error.obj
 0001:00000054       _fz_rethrowimp             00401054 f   base_error.obj
 0001:000000a8       _fz_catchimp               004010a8 f   base_error.obj
 0001:000000fc       _fz_malloc                 004010fc f   base_memory.obj
 0001:0000012e       _fz_realloc                0040112e f   base_memory.obj
 0001:00000165       _fz_readimp                00401165 f   stm_read.obj
 0001:00000344       _fz_readerror              00401344 f   stm_read.obj
 0001:00000370       _fz_readbytex              00401370 f   stm_read.obj
 0001:000003c9       _fz_peekbytex              004013c9 f   stm_read.obj
 0001:0000041d       _fz_newbuffer              0040141d f   stm_buffer.obj
 0001:0000049a       _fz_dropbuffer             0040149a f   stm_buffer.obj
 0001:000004b5       _fz_growbuffer             004014b5 f   stm_buffer.obj
 0001:00000532       _fz_rewindbuffer           00401532 f   stm_buffer.obj
 0001:00000578       _fz_process                00401578 f   stm_filter.obj
 0001:00000624       _fz_dropstream             00401624 f   stm_open.obj
 0001:0000069d       _fz_openrfile              0040169d f   stm_open.obj
 0001:0000075e       _fz_strlcpy                0040175e f   base_string.obj
 0001:00000cf7       _pdf_lex                   00401cf7 f   cmapdump.obj
 0001:00000f80       _pdf_newcmap               00401f80 f   cmapdump.obj
 0001:00000ffb       _pdf_dropcmap              00401ffb f   cmapdump.obj
 0001:0000117a       _pdf_maprangetorange       0040217a f   cmapdump.obj
 0001:000011c2       _pdf_maponetomany          004021c2 f   cmapdump.obj
 0001:000012b8       _pdf_sortcmap              004022b8 f   cmapdump.obj
 0001:00002273       _pdf_parsecmap             00403273 f   cmapdump.obj
 0001:00002538       _main                      00403538 f   cmapdump.obj
 0001:0000297f       @__security_check_cookie@4 0040397f f   LIBCMT:secchk.obj
 0001:0000298e       ___iob_func                0040398e f   LIBCMT:_file.obj
 0001:00002994       ___initstdio               00403994 f   LIBCMT:_file.obj
 0001:00002a45       ___endstdio                00403a45 f   LIBCMT:_file.obj
 0001:00002a65       __lock_file                00403a65 f   LIBCMT:_file.obj
 0001:00002aa1       __lock_file2               00403aa1 f   LIBCMT:_file.obj
 0001:00002acf       __unlock_file              00403acf f   LIBCMT:_file.obj
 0001:00002b05       __unlock_file2             00403b05 f   LIBCMT:_file.obj
 0001:00002b2f       _fprintf                   00403b2f f   LIBCMT:fprintf.obj
 0001:00002c7e       _vfprintf_helper           00403c7e f   LIBCMT:vfprintf.obj
 0001:00002dcc       _vfprintf                  00403dcc f   LIBCMT:vfprintf.obj
 0001:00002de8       _free                      00403de8 f   LIBCMT:free.obj
 0001:00002e76       _V6_HeapAlloc              00403e76 f   LIBCMT:malloc.obj
 0001:00002ec5       _malloc                    00403ec5 f   LIBCMT:malloc.obj
 0001:00002f88       _realloc                   00403f88 f   LIBCMT:realloc.obj
 0001:000031a3       __get_sys_err_msg          004041a3 f i LIBCMT:strerror.obj
 0001:000031c6       _strerror                  004041c6 f   LIBCMT:strerror.obj
 0001:0000322d       __get_errno_from_oserr     0040422d f   LIBCMT:dosmap.obj
 0001:00003268       __errno                    00404268 f   LIBCMT:dosmap.obj
 0001:0000327b       ___doserrno                0040427b f   LIBCMT:dosmap.obj
 0001:0000328e       __dosmaperr                0040428e f   LIBCMT:dosmap.obj
 0001:000032b0       _memmove                   004042b0 f   LIBCMT:memmove.obj
 0001:00003620       _strpbrk                   00404620 f   LIBCMT:strpbrk.obj
 0001:00003660       _strrchr                   00404660 f   LIBCMT:strrchr.obj
 0001:00003750       _qsort                     00404750 f   LIBCMT:qsort.obj
 0001:00003a10       _strchr                    00404a10 f   LIBCMT:strchr.obj
 0001:00003a16       ___from_strstr_to_strchr   00404a16     LIBCMT:strchr.obj
 0001:00003ace       _atol                      00404ace f   LIBCMT:atox.obj
 0001:00003adf       _atoi                      00404adf f   LIBCMT:atox.obj
 0001:00003ae4       __get_printf_count_output  00404ae4 f   LIBCMT:printf.obj
 0001:00003afa       __fsopen                   00404afa f   LIBCMT:fopen.obj
 0001:00003bbe       _fopen                     00404bbe f   LIBCMT:fopen.obj
 0001:00003dec       _mainCRTStartup            00404dec f   LIBCMT:crt0.obj
 0001:00003df6       ___report_gsfailure        00404df6 f   LIBCMT:gs_report.obj
 0001:00003efa       __ioinit                   00404efa f   LIBCMT:ioinit.obj
 0001:0000413a       __malloc_crt               0040513a f   LIBCMT:crtheap.obj
 0001:0000417a       __calloc_crt               0040517a f   LIBCMT:crtheap.obj
 0001:000041c2       __realloc_crt              004051c2 f   LIBCMT:crtheap.obj
 0001:0000420d       __fcloseall                0040520d f   LIBCMT:closeall.obj
 0001:000042ac       __amsg_exit                004052ac f   LIBCMT:crt0dat.obj
 0001:000042d0       ___crtCorExitProcess       004052d0 f   LIBCMT:crt0dat.obj
 0001:000042f6       ___crtExitProcess          004052f6 f   LIBCMT:crt0dat.obj
 0001:0000430b       __lockexit                 0040530b f   LIBCMT:crt0dat.obj
 0001:00004314       __unlockexit               00405314 f   LIBCMT:crt0dat.obj
 0001:00004335       __initterm_e               00405335 f   LIBCMT:crt0dat.obj
 0001:00004355       __get_osplatform           00405355 f   LIBCMT:crt0dat.obj
 0001:0000438c       __get_winmajor             0040538c f   LIBCMT:crt0dat.obj
 0001:000043c8       __cinit                    004053c8 f   LIBCMT:crt0dat.obj
 0001:0000453c       _exit                      0040553c f   LIBCMT:crt0dat.obj
 0001:0000454d       __exit                     0040554d f   LIBCMT:crt0dat.obj
 0001:0000455e       __cexit                    0040555e f   LIBCMT:crt0dat.obj
 0001:0000456d       __c_exit                   0040556d f   LIBCMT:crt0dat.obj
 0001:0000457c       __init_pointers            0040557c f   LIBCMT:crt0dat.obj
 0001:000045c8       __flush                    004055c8 f   LIBCMT:fflush.obj
 0001:0000462a       __fflush_nolock            0040562a f   LIBCMT:fflush.obj
 0001:00004746       __flushall                 00405746 f   LIBCMT:fflush.obj
 0001:0000474f       __mtinitlocks              0040574f f   LIBCMT:mlock.obj
 0001:00004798       __mtdeletelocks            00405798 f   LIBCMT:mlock.obj
 0001:000047ed       __unlock                   004057ed f   LIBCMT:mlock.obj
 0001:00004802       __mtinitlocknum            00405802 f   LIBCMT:mlock.obj
 0001:000048c5       __lock                     004058c5 f   LIBCMT:mlock.obj
 0001:000048f6       __stbuf                    004058f6 f   LIBCMT:_sftbuf.obj
 0001:0000498c       __ftbuf                    0040598c f   LIBCMT:_sftbuf.obj
 0001:000049bb       ??0_LocaleUpdate@@QAE@PAUlocaleinfo_struct@@@Z 004059bb f i LIBCMT:output.obj
 0001:00004ade       __output_l                 00405ade f   LIBCMT:output.obj
 0001:00005472       __fileno                   00406472 f   LIBCMT:fileno.obj
 0001:0000549f       __initp_misc_invarg        0040649f f   LIBCMT:invarg.obj
 0001:000054a9       __invoke_watson            004064a9 f   LIBCMT:invarg.obj
 0001:000055a5       __invalid_parameter        004065a5 f   LIBCMT:invarg.obj
 0001:000055cc       __SEH_prolog4              004065cc f   LIBCMT:sehprolg4.obj
 0001:00005611       __SEH_epilog4              00406611 f   LIBCMT:sehprolg4.obj
 0001:00005630       __except_handler4          00406630 f   LIBCMT:chandler4.obj
 0001:000057c6       ___heap_select             004067c6 f   LIBCMT:heapinit.obj
 0001:00005821       __heap_init                00406821 f   LIBCMT:heapinit.obj
 0001:0000587b       ___sbh_heap_init           0040687b f   LIBCMT:sbheap.obj
 0001:000058c3       ___sbh_find_block          004068c3 f   LIBCMT:sbheap.obj
 0001:000058ee       ___sbh_free_block          004068ee f   LIBCMT:sbheap.obj
 0001:00005c02       ___sbh_alloc_new_region    00406c02 f   LIBCMT:sbheap.obj
 0001:00005cb2       ___sbh_alloc_new_group     00406cb2 f   LIBCMT:sbheap.obj
 0001:00005db8       ___sbh_resize_block        00406db8 f   LIBCMT:sbheap.obj
 0001:00006097       ___sbh_alloc_block         00407097 f   LIBCMT:sbheap.obj
 0001:0000637a       __NMSG_WRITE               0040737a f   LIBCMT:crt0msg.obj
 0001:0000651a       __FF_MSGBANNER             0040751a f   LIBCMT:crt0msg.obj
 0001:00006553       __initp_heap_handler       00407553 f   LIBCMT:handler.obj
 0001:0000655d       __callnewh                 0040755d f   LIBCMT:handler.obj
 0001:00006580       _memcpy                    00407580 f   LIBCMT:memcpy.obj
 0001:000068f0       _memset                    004078f0 f   LIBCMT:memset.obj
 0001:0000696a       __msize                    0040796a f   LIBCMT:msize.obj
 0001:00006a0d       ___sys_nerr                00407a0d f   LIBCMT:syserr.obj
 0001:00006a13       ___sys_errlist             00407a13 f   LIBCMT:syserr.obj
 0001:00006a19       _strcpy_s                  00407a19 f   LIBCMT:strcpy_s.obj
 0001:00006aea       __encode_pointer           00407aea f   LIBCMT:tidtable.obj
 0001:00006b58       __encoded_null             00407b58 f   LIBCMT:tidtable.obj
 0001:00006b61       __decode_pointer           00407b61 f   LIBCMT:tidtable.obj
 0001:00006bcf       ___crtTlsAlloc@4           00407bcf f   LIBCMT:tidtable.obj
 0001:00006bd8       ___set_flsgetvalue         00407bd8 f   LIBCMT:tidtable.obj
 0001:00006c0a       __mtterm                   00407c0a f   LIBCMT:tidtable.obj
 0001:00006c47       __initptd                  00407c47 f   LIBCMT:tidtable.obj
 0001:00006d06       __getptd_noexit            00407d06 f   LIBCMT:tidtable.obj
 0001:00006d7d       __getptd                   00407d7d f   LIBCMT:tidtable.obj
 0001:00006d95       __freefls@4                00407d95 f   LIBCMT:tidtable.obj
 0001:00006eb6       __mtinit                   00407eb6 f   LIBCMT:tidtable.obj
 0001:0000703a       _strncpy_s                 0040803a f   LIBCMT:strncpy_s.obj
 0001:00007174       __VEC_memcpy               00408174 f   LIBCMT:p4_memcpy.obj
 0001:00007257       __sse2_mathfcns_init       00408257 f   LIBCMT:mathfcns.obj
 0001:0000726b       __write_nolock             0040826b f   LIBCMT:write.obj
 0001:00007831       __write                    00408831 f   LIBCMT:write.obj
 0001:0000790d       __lseeki64_nolock          0040890d f   LIBCMT:lseeki64.obj
 0001:00007990       __lseeki64                 00408990 f   LIBCMT:lseeki64.obj
 0001:00007aa9       __set_osfhnd               00408aa9 f   LIBCMT:osfinfo.obj
 0001:00007b26       __free_osfhnd              00408b26 f   LIBCMT:osfinfo.obj
 0001:00007ba7       __get_osfhandle            00408ba7 f   LIBCMT:osfinfo.obj
 0001:00007c18       ___lock_fhandle            00408c18 f   LIBCMT:osfinfo.obj
 0001:00007cb8       __unlock_fhandle           00408cb8 f   LIBCMT:osfinfo.obj
 0001:00007cda       __alloc_osfhnd             00408cda f   LIBCMT:osfinfo.obj
 0001:00007e79       __chsize_nolock            00408e79 f   LIBCMT:chsize.obj
 0001:0000802d       __read_nolock              0040902d f   LIBCMT:read.obj
 0001:000085ee       __read                     004095ee f   LIBCMT:read.obj
 0001:000085ee       _read                      004095ee f   LIBCMT:read.obj
 0001:000086eb       __close_nolock             004096eb f   LIBCMT:close.obj
 0001:0000877f       __close                    0040977f f   LIBCMT:close.obj
 0001:0000877f       _close                     0040977f f   LIBCMT:close.obj
 0001:0000884c       __lseek_nolock             0040984c f   LIBCMT:lseek.obj
 0001:000088be       __setmode_nolock           004098be f   LIBCMT:setmode.obj
 0001:0000897a       __get_fmode                0040997a f   LIBCMT:setmode.obj
 0001:00008bd9       _strtol                    00409bd9 f   LIBCMT:strtol.obj
 0001:00008c02       __openfile                 00409c02 f   LIBCMT:_open.obj
 0001:00008ea2       __getstream                00409ea2 f   LIBCMT:stream.obj
 0001:00008fd4       __local_unwind4            00409fd4 f   LIBCMT:exsup4.obj
 0001:000090aa       __seh_longjmp_unwind4@4    0040a0aa f   LIBCMT:exsup4.obj
 0001:000090c6       @_EH4_CallFilterFunc@8     0040a0c6 f   LIBCMT:exsup4.obj
 0001:000090dd       @_EH4_TransferToHandler@8  0040a0dd f   LIBCMT:exsup4.obj
 0001:000090f6       @_EH4_GlobalUnwind@4       0040a0f6 f   LIBCMT:exsup4.obj
 0001:00009110       @_EH4_LocalUnwind@16       0040a110 f   LIBCMT:exsup4.obj
 0001:00009127       ?__CxxUnhandledExceptionFilter@@YGJPAU_EXCEPTION_POINTERS@@@Z 0040a127 f   LIBCMT:unhandld.obj
 0001:00009164       ___CxxSetUnhandledExceptionFilter 0040a164 f   LIBCMT:unhandld.obj
 0001:00009172       __initp_misc_winxfltr      0040a172 f   LIBCMT:winxfltr.obj
 0001:00009173       __XcptFilter               0040a173 f   LIBCMT:winxfltr.obj
 0001:000092d1       __setenvp                  0040a2d1 f   LIBCMT:stdenvp.obj
 0001:00009544       __setargv                  0040a544 f   LIBCMT:stdargv.obj
 0001:000095fd       ___crtGetEnvironmentStringsA 0040a5fd f   LIBCMT:a_env.obj
 0001:00009732       __RTC_Initialize           0040a732 f   LIBCMT:initsect.obj
 0001:00009756       __RTC_Terminate            0040a756 f   LIBCMT:initsect.obj
 0001:0000977a       ___security_init_cookie    0040a77a f   LIBCMT:gs_support.obj
 0001:0000980e       __crt_debugger_hook        0040a80e f   LIBCMT:dbghook.obj
 0001:00009816       __initp_misc_initcrit      0040a816 f   LIBCMT:initcrit.obj
 0001:00009830       ___crtInitCritSecAndSpinCount 0040a830 f   LIBCMT:initcrit.obj
 0001:000098f5       __calloc_impl              0040a8f5 f   LIBCMT:calloc.obj
 0001:00009a13       __fclose_nolock            0040aa13 f   LIBCMT:fclose.obj
 0001:00009a85       _fclose                    0040aa85 f   LIBCMT:fclose.obj
 0001:00009bba       ___onexitinit              0040abba f   LIBCMT:onexit.obj
 0001:00009be9       __onexit                   0040abe9 f   LIBCMT:onexit.obj
 0001:00009c25       _atexit                    0040ac25 f   LIBCMT:onexit.obj
 0001:00009c37       __initp_misc_cfltcvt_tab   0040ac37 f   LIBCMT:cmiscdat.obj
 0001:00009c60       __ValidateImageBase        0040ac60 f   LIBCMT:pesect.obj
 0001:00009c90       __FindPESection            0040ac90 f   LIBCMT:pesect.obj
 0001:00009ce0       __IsNonwritableInCurrentImage 0040ace0 f   LIBCMT:pesect.obj
 0001:00009d9b       ?terminate@@YAXXZ          0040ad9b f   LIBCMT:hooks.obj
 0001:00009dd4       __initp_eh_hooks           0040add4 f   LIBCMT:hooks.obj
 0001:00009de5       __initp_misc_winsig        0040ade5 f   LIBCMT:winsig.obj
 0001:00009e32       ___get_sigabrt             0040ae32 f   LIBCMT:winsig.obj
 0001:00009e3f       _raise                     0040ae3f f   LIBCMT:winsig.obj
 0001:00009fef       __initp_misc_rand_s        0040afef f   LIBCMT:rand_s.obj
 0001:00009ff9       __initp_misc_purevirt      0040aff9 f   LIBCMT:inithelp.obj
 0001:0000a003       __commit                   0040b003 f   LIBCMT:commit.obj
 0001:0000a0e4       __isatty                   0040b0e4 f   LIBCMT:isatty.obj
 0001:0000a350       ___updatetmbcinfo          0040b350 f   LIBCMT:mbctype.obj
 0001:0000a46e       __setmbcp_nolock           0040b46e f   LIBCMT:mbctype.obj
 0001:0000a647       __setmbcp                  0040b647 f   LIBCMT:mbctype.obj
 0001:0000a7e1       ___initmbctable            0040b7e1 f   LIBCMT:mbctype.obj
 0001:0000a7ff       ___freetlocinfo            0040b7ff f   LIBCMT:setlocal.obj
 0001:0000a93f       ___addlocaleref            0040b93f f   LIBCMT:setlocal.obj
 0001:0000a9c5       ___removelocaleref         0040b9c5 f   LIBCMT:setlocal.obj
 0001:0000aa8f       ___updatetlocinfo          0040ba8f f   LIBCMT:setlocal.obj
 0001:0000ab05       __flsbuf                   0040bb05 f   LIBCMT:_flsbuf.obj
 0001:0000ac70       _strlen                    0040bc70 f   LIBCMT:strlen.obj
 0001:0000acfb       __wctomb_s_l               0040bcfb f   LIBCMT:wctomb.obj
 0001:0000ae5a       _wctomb_s                  0040be5a f   LIBCMT:wctomb.obj
 0001:0000ae75       __isleadbyte_l             0040be75 f i LIBCMT:_wctype.obj
 0001:0000aeab       _isleadbyte                0040beab f i LIBCMT:_wctype.obj
 0001:0000aec0       __aulldvrm                 0040bec0 f   LIBCMT:ulldvrm.obj
 0001:0000af55       ___crtMessageBoxA          0040bf55 f   LIBCMT:crtmbox.obj
 0001:0000b112       _strcat_s                  0040c112 f   LIBCMT:strcat_s.obj
 0001:0000b183       __set_error_mode           0040c183 f   LIBCMT:errmode.obj
 0001:0000b220       __VEC_memzero              0040c220 f   LIBCMT:p4_memset.obj
 0001:0000b2b0       _strcmp                    0040c2b0 f   LIBCMT:strcmp.obj
 0001:0000b388       __get_sse2_info            0040c388 f   LIBCMT:cpu_disp.obj
 0001:0000b3e8       ___sse2_available_init     0040c3e8 f   LIBCMT:cpu_disp.obj
 0001:0000b3f5       __putwch_nolock            0040c3f5 f   LIBCMT:putwch.obj
 0001:0000b4b7       __mbtowc_l                 0040c4b7 f   LIBCMT:mbtowc.obj
 0001:0000b5ca       _mbtowc                    0040c5ca f   LIBCMT:mbtowc.obj
 0001:0000b5e1       __isctype_l                0040c5e1 f   LIBCMT:isctype.obj
 0001:0000b6a0       __allmul                   0040c6a0 f   LIBCMT:llmul.obj
 0001:0000be2d       __open                     0040ce2d f   LIBCMT:open.obj
 0001:0000be2d       _open                      0040ce2d f   LIBCMT:open.obj
 0001:0000bee3       __sopen_helper             0040cee3 f   LIBCMT:open.obj
 0001:0000bfaf       __sopen_s                  0040cfaf f   LIBCMT:open.obj
 0001:0000bfcd       __mbsicmp_l                0040cfcd f   LIBCMT:mbsicmp.obj
 0001:0000c1e7       __mbsicmp                  0040d1e7 f   LIBCMT:mbsicmp.obj
 0001:0000c1fa       __mbsnbcmp_l               0040d1fa f   LIBCMT:mbsnbcmp.obj
 0001:0000c363       __mbsnbcmp                 0040d363 f   LIBCMT:mbsnbcmp.obj
 0001:0000c37c       __global_unwind2           0040d37c f   LIBCMT:exsup.obj
 0001:0000c3e1       __local_unwind2            0040d3e1 f   LIBCMT:exsup.obj
 0001:0000c465       __abnormal_termination     0040d465 f   LIBCMT:exsup.obj
 0001:0000c488       __NLG_Notify1              0040d488 f   LIBCMT:exsup.obj
 0001:0000c491       __NLG_Notify               0040d491 f   LIBCMT:exsup.obj
 0001:0000c4a8       __NLG_Dispatch             0040d4a8     LIBCMT:exsup.obj
 0001:0000c4a8       __NLG_Dispatch2            0040d4a8     LIBCMT:exsup.obj
 0001:0000c4b0       __NLG_Call                 0040d4b0 f   LIBCMT:exsup.obj
 0001:0000c4b2       __NLG_Return2              0040d4b2     LIBCMT:exsup.obj
 0001:0000c504       __ismbblead                0040d504 f   LIBCMT:ismbbyte.obj
 0001:0000c517       __freebuf                  0040d517 f   LIBCMT:_freebuf.obj
 0001:0000c543       __fptrap                   0040d543 f   LIBCMT:crt0fp.obj
 0001:0000c54c       _abort                     0040d54c f   LIBCMT:abort.obj
 0001:0000c63f       __freea                    0040d63f f i LIBCMT:w_loc.obj
 0001:0000c9fc       ___crtLCMapStringA         0040d9fc f   LIBCMT:a_map.obj
 0001:0000cbf7       ___crtGetStringTypeA       0040dbf7 f   LIBCMT:a_str.obj
 0001:0000cc37       ___free_lc_time            0040dc37 f   LIBCMT:inittime.obj
 0001:0000cdc7       ___free_lconv_num          0040ddc7 f   LIBCMT:initnum.obj
 0001:0000ce07       ___free_lconv_mon          0040de07 f   LIBCMT:initmon.obj
 0001:0000ce90       _strcspn                   0040de90 f   LIBCMT:strcspn.obj
 0001:0000ced6       _strncmp                   0040ded6 f   LIBCMT:strncmp.obj
 0001:0000cf94       __getbuf                   0040df94 f   LIBCMT:_getbuf.obj
 0001:0000cfd8       ___initconout              0040dfd8 f   LIBCMT:initcon.obj
 0001:0000cff7       ___termcon                 0040dff7 f   LIBCMT:initcon.obj
 0001:0000d024       ___ascii_stricmp           0040e024 f   LIBCMT:stricmp.obj
 0001:0000d059       __stricmp_l                0040e059 f   LIBCMT:stricmp.obj
 0001:0000d130       __alloca_probe_16          0040e130 f   LIBCMT:alloca16.obj
 0001:0000d146       __alloca_probe_8           0040e146     LIBCMT:alloca16.obj
 0001:0000d15c       ___ansicp                  0040e15c f   LIBCMT:convrtcp.obj
 0001:0000d1a3       ___convertcp               0040e1a3 f   LIBCMT:convrtcp.obj
 0001:0000d355       __tolower_l                0040e355 f   LIBCMT:tolower.obj
 0001:0000d470       __chkstk                   0040e470 f   LIBCMT:chkstk.obj
 0001:0000d470       __alloca_probe             0040e470     LIBCMT:chkstk.obj
 0001:0000d4a0       ___ascii_strnicmp          0040e4a0 f   LIBCMT:_strnicm.obj
 0001:0000d502       _RtlUnwind@16              0040e502 f   kernel32:KERNEL32.dll
 0002:00000000       __imp__EnterCriticalSection@4 0040f000     kernel32:KERNEL32.dll
 0002:00000004       __imp__LeaveCriticalSection@4 0040f004     kernel32:KERNEL32.dll
 0002:00000008       __imp__GetLastError@0      0040f008     kernel32:KERNEL32.dll
 0002:0000000c       __imp__HeapFree@12         0040f00c     kernel32:KERNEL32.dll
 0002:00000010       __imp__HeapAlloc@12        0040f010     kernel32:KERNEL32.dll
 0002:00000014       __imp__HeapReAlloc@16      0040f014     kernel32:KERNEL32.dll
 0002:00000018       __imp__CloseHandle@4       0040f018     kernel32:KERNEL32.dll
 0002:0000001c       __imp__GetFileType@4       0040f01c     kernel32:KERNEL32.dll
 0002:00000020       __imp__GetCommandLineA@0   0040f020     kernel32:KERNEL32.dll
 0002:00000024       __imp__GetVersionExA@4     0040f024     kernel32:KERNEL32.dll
 0002:00000028       __imp__GetProcessHeap@0    0040f028     kernel32:KERNEL32.dll
 0002:0000002c       __imp__TerminateProcess@8  0040f02c     kernel32:KERNEL32.dll
 0002:00000030       __imp__GetCurrentProcess@0 0040f030     kernel32:KERNEL32.dll
 0002:00000034       __imp__UnhandledExceptionFilter@4 0040f034     kernel32:KERNEL32.dll
 0002:00000038       __imp__SetUnhandledExceptionFilter@4 0040f038     kernel32:KERNEL32.dll
 0002:0000003c       __imp__IsDebuggerPresent@0 0040f03c     kernel32:KERNEL32.dll
 0002:00000040       __imp__SetHandleCount@4    0040f040     kernel32:KERNEL32.dll
 0002:00000044       __imp__GetStdHandle@4      0040f044     kernel32:KERNEL32.dll
 0002:00000048       __imp__GetStartupInfoA@4   0040f048     kernel32:KERNEL32.dll
 0002:0000004c       __imp__DeleteCriticalSection@4 0040f04c     kernel32:KERNEL32.dll
 0002:00000050       __imp__Sleep@4             0040f050     kernel32:KERNEL32.dll
 0002:00000054       __imp__GetProcAddress@8    0040f054     kernel32:KERNEL32.dll
 0002:00000058       __imp__GetModuleHandleA@4  0040f058     kernel32:KERNEL32.dll
 0002:0000005c       __imp__ExitProcess@4       0040f05c     kernel32:KERNEL32.dll
 0002:00000060       __imp__HeapDestroy@4       0040f060     kernel32:KERNEL32.dll
 0002:00000064       __imp__HeapCreate@12       0040f064     kernel32:KERNEL32.dll
 0002:00000068       __imp__VirtualFree@12      0040f068     kernel32:KERNEL32.dll
 0002:0000006c       __imp__VirtualAlloc@16     0040f06c     kernel32:KERNEL32.dll
 0002:00000070       __imp__WriteFile@20        0040f070     kernel32:KERNEL32.dll
 0002:00000074       __imp__GetModuleFileNameA@12 0040f074     kernel32:KERNEL32.dll
 0002:00000078       __imp__HeapSize@12         0040f078     kernel32:KERNEL32.dll
 0002:0000007c       __imp__TlsGetValue@4       0040f07c     kernel32:KERNEL32.dll
 0002:00000080       __imp__TlsAlloc@0          0040f080     kernel32:KERNEL32.dll
 0002:00000084       __imp__TlsSetValue@8       0040f084     kernel32:KERNEL32.dll
 0002:00000088       __imp__TlsFree@4           0040f088     kernel32:KERNEL32.dll
 0002:0000008c       __imp__InterlockedIncrement@4 0040f08c     kernel32:KERNEL32.dll
 0002:00000090       __imp__SetLastError@4      0040f090     kernel32:KERNEL32.dll
 0002:00000094       __imp__GetCurrentThreadId@0 0040f094     kernel32:KERNEL32.dll
 0002:00000098       __imp__InterlockedDecrement@4 0040f098     kernel32:KERNEL32.dll
 0002:0000009c       __imp__WideCharToMultiByte@32 0040f09c     kernel32:KERNEL32.dll
 0002:000000a0       __imp__GetConsoleCP@0      0040f0a0     kernel32:KERNEL32.dll
 0002:000000a4       __imp__GetConsoleMode@8    0040f0a4     kernel32:KERNEL32.dll
 0002:000000a8       __imp__SetFilePointer@16   0040f0a8     kernel32:KERNEL32.dll
 0002:000000ac       __imp__SetStdHandle@8      0040f0ac     kernel32:KERNEL32.dll
 0002:000000b0       __imp__SetEndOfFile@4      0040f0b0     kernel32:KERNEL32.dll
 0002:000000b4       __imp__MultiByteToWideChar@24 0040f0b4     kernel32:KERNEL32.dll
 0002:000000b8       __imp__ReadFile@20         0040f0b8     kernel32:KERNEL32.dll
 0002:000000bc       __imp__RtlUnwind@16        0040f0bc     kernel32:KERNEL32.dll
 0002:000000c0       __imp__FreeEnvironmentStringsA@4 0040f0c0     kernel32:KERNEL32.dll
 0002:000000c4       __imp__GetEnvironmentStrings@0 0040f0c4     kernel32:KERNEL32.dll
 0002:000000c8       __imp__FreeEnvironmentStringsW@4 0040f0c8     kernel32:KERNEL32.dll
 0002:000000cc       __imp__GetEnvironmentStringsW@0 0040f0cc     kernel32:KERNEL32.dll
 0002:000000d0       __imp__QueryPerformanceCounter@4 0040f0d0     kernel32:KERNEL32.dll
 0002:000000d4       __imp__GetTickCount@0      0040f0d4     kernel32:KERNEL32.dll
 0002:000000d8       __imp__GetCurrentProcessId@0 0040f0d8     kernel32:KERNEL32.dll
 0002:000000dc       __imp__GetSystemTimeAsFileTime@4 0040f0dc     kernel32:KERNEL32.dll
 0002:000000e0       __imp__InitializeCriticalSection@4 0040f0e0     kernel32:KERNEL32.dll
 0002:000000e4       __imp__LoadLibraryA@4      0040f0e4     kernel32:KERNEL32.dll
 0002:000000e8       __imp__FlushFileBuffers@4  0040f0e8     kernel32:KERNEL32.dll
 0002:000000ec       __imp__GetCPInfo@8         0040f0ec     kernel32:KERNEL32.dll
 0002:000000f0       __imp__GetACP@0            0040f0f0     kernel32:KERNEL32.dll
 0002:000000f4       __imp__GetOEMCP@0          0040f0f4     kernel32:KERNEL32.dll
 0002:000000f8       __imp__IsValidCodePage@4   0040f0f8     kernel32:KERNEL32.dll
 0002:000000fc       __imp__WriteConsoleA@20    0040f0fc     kernel32:KERNEL32.dll
 0002:00000100       __imp__GetConsoleOutputCP@0 0040f100     kernel32:KERNEL32.dll
 0002:00000104       __imp__WriteConsoleW@20    0040f104     kernel32:KERNEL32.dll
 0002:00000108       __imp__CreateFileA@28      0040f108     kernel32:KERNEL32.dll
 0002:0000010c       __imp__GetLocaleInfoA@16   0040f10c     kernel32:KERNEL32.dll
 0002:00000110       __imp__LCMapStringA@24     0040f110     kernel32:KERNEL32.dll
 0002:00000114       __imp__LCMapStringW@24     0040f114     kernel32:KERNEL32.dll
 0002:00000118       __imp__GetStringTypeA@20   0040f118     kernel32:KERNEL32.dll
 0002:0000011c       __imp__GetStringTypeW@16   0040f11c     kernel32:KERNEL32.dll
 0002:00000120       \177KERNEL32_NULL_THUNK_DATA 0040f120     kernel32:KERNEL32.dll
 0002:00000124       ___xc_a                    0040f124     LIBCMT:crt0init.obj
 0002:00000128       ___xc_z                    0040f128     LIBCMT:crt0init.obj
 0002:0000012c       ___xi_a                    0040f12c     LIBCMT:crt0init.obj
 0002:00000148       ___xi_z                    0040f148     LIBCMT:crt0init.obj
 0002:0000014c       ___xp_a                    0040f14c     LIBCMT:crt0init.obj
 0002:00000158       ___xp_z                    0040f158     LIBCMT:crt0init.obj
 0002:0000015c       ___xt_a                    0040f15c     LIBCMT:crt0init.obj
 0002:00000160       ___xt_z                    0040f160     LIBCMT:crt0init.obj
 0002:00000190       ??_C@_0EA@FCLIIPNN@Visual?5C?$CL?$CL?5CRT?3?5Not?5enough?5memor@ 0040f190     LIBCMT:strerror.obj
 0002:000001d8       ??_C@_0P@MIGLKIOC@CorExitProcess?$AA@ 0040f1d8     LIBCMT:crt0dat.obj
 0002:000001e8       ??_C@_0M@MBOPBNBK@mscoree?4dll?$AA@ 0040f1e8     LIBCMT:crt0dat.obj
 0002:000001f4       ??_C@_1O@CEDCILHN@?$AA?$CI?$AAn?$AAu?$AAl?$AAl?$AA?$CJ?$AA?$AA@ 0040f1f4     LIBCMT:output.obj
 0002:00000204       ??_C@_06OJHGLDPL@?$CInull?$CJ?$AA@ 0040f204     LIBCMT:output.obj
 0002:00000210       ___lookuptable             0040f210     LIBCMT:output.obj
 0002:00000270       ___lookuptable_s           0040f270     LIBCMT:outputs.obj
 0002:000002cc       ??_C@_0P@GGKDKEEG@runtime?5error?5?$AA@ 0040f2cc     LIBCMT:crt0msg.obj
 0002:000002dc       ??_C@_02PCIJFNDE@?$AN?6?$AA@ 0040f2dc     LIBCMT:crt0msg.obj
 0002:000002e0       ??_C@_0O@MJNIPGOH@TLOSS?5error?$AN?6?$AA@ 0040f2e0     LIBCMT:crt0msg.obj
 0002:000002f0       ??_C@_0N@BONNPDHF@SING?5error?$AN?6?$AA@ 0040f2f0     LIBCMT:crt0msg.obj
 0002:00000300       ??_C@_0P@MBDAJNE@DOMAIN?5error?$AN?6?$AA@ 0040f300     LIBCMT:crt0msg.obj
 0002:00000310       ??_C@_0JL@DFDOOABL@R6034?$AN?6An?5application?5has?5made?5a@ 0040f310     LIBCMT:crt0msg.obj
 0002:000003b0       ??_C@_0PH@EPAFIJ@R6033?$AN?6?9?5Attempt?5to?5use?5MSIL?5cod@ 0040f3b0     LIBCMT:crt0msg.obj
 0002:000004a8       ??_C@_0DD@BKEEABMM@R6032?$AN?6?9?5not?5enough?5space?5for?5lo@ 0040f4a8     LIBCMT:crt0msg.obj
 0002:000004e0       ??_C@_0GD@OFKILIED@R6031?$AN?6?9?5Attempt?5to?5initialize?5t@ 0040f4e0     LIBCMT:crt0msg.obj
 0002:00000544       ??_C@_0BP@LPMHJOKI@R6030?$AN?6?9?5CRT?5not?5initialized?$AN?6?$AA@ 0040f544     LIBCMT:crt0msg.obj
 0002:00000564       ??_C@_0CF@KJDAIALP@R6028?$AN?6?9?5unable?5to?5initialize?5he@ 0040f564     LIBCMT:crt0msg.obj
 0002:0000058c       ??_C@_0DF@GAKBPDFP@R6027?$AN?6?9?5not?5enough?5space?5for?5lo@ 0040f58c     LIBCMT:crt0msg.obj
 0002:000005c4       ??_C@_0DF@IBLNNAIG@R6026?$AN?6?9?5not?5enough?5space?5for?5st@ 0040f5c4     LIBCMT:crt0msg.obj
 0002:000005fc       ??_C@_0CG@IOHKGFNJ@R6025?$AN?6?9?5pure?5virtual?5function?5c@ 0040f5fc     LIBCMT:crt0msg.obj
 0002:00000624       ??_C@_0DF@JIJJFJDC@R6024?$AN?6?9?5not?5enough?5space?5for?5_o@ 0040f624     LIBCMT:crt0msg.obj
 0002:0000065c       ??_C@_0CJ@EGEJHFME@R6019?$AN?6?9?5unable?5to?5open?5console?5@ 0040f65c     LIBCMT:crt0msg.obj
 0002:00000688       ??_C@_0CB@GNHNIELH@R6018?$AN?6?9?5unexpected?5heap?5error?$AN?6@ 0040f688     LIBCMT:crt0msg.obj
 0002:000006ac       ??_C@_0CN@FOLDKNG@R6017?$AN?6?9?5unexpected?5multithread?5@ 0040f6ac     LIBCMT:crt0msg.obj
 0002:000006dc       ??_C@_0CM@FAHFJNHO@R6016?$AN?6?9?5not?5enough?5space?5for?5th@ 0040f6dc     LIBCMT:crt0msg.obj
 0002:00000708       ??_C@_0JG@LBKMGKLD@?$AN?6This?5application?5has?5requested@ 0040f708     LIBCMT:crt0msg.obj
 0002:000007a0       ??_C@_0CM@FLCNIPKK@R6009?$AN?6?9?5not?5enough?5space?5for?5en@ 0040f7a0     LIBCMT:crt0msg.obj
 0002:000007cc       ??_C@_0CK@KMMJOAPP@R6008?$AN?6?9?5not?5enough?5space?5for?5ar@ 0040f7cc     LIBCMT:crt0msg.obj
 0002:000007f8       ??_C@_0CN@LEKKICBM@R6002?$AN?6?9?5floating?5point?5support?5@ 0040f7f8     LIBCMT:crt0msg.obj
 0002:00000828       ??_C@_0CF@GOGNBNAK@Microsoft?5Visual?5C?$CL?$CL?5Runtime?5Lib@ 0040f828     LIBCMT:crt0msg.obj
 0002:00000850       ??_C@_02PHMGELLB@?6?6?$AA@ 0040f850     LIBCMT:crt0msg.obj
 0002:00000854       ??_C@_03KHICJKCI@?4?4?4?$AA@ 0040f854     LIBCMT:crt0msg.obj
 0002:00000858       ??_C@_0BH@DNAGHKFM@?$DMprogram?5name?5unknown?$DO?$AA@ 0040f858     LIBCMT:crt0msg.obj
 0002:00000870       ??_C@_0BK@OFGJDLJJ@Runtime?5Error?$CB?6?6Program?3?5?$AA@ 0040f870     LIBCMT:crt0msg.obj
 0002:0000088c       ??_C@_0BG@KLEAJEFJ@Illegal?5byte?5sequence?$AA@ 0040f88c     LIBCMT:syserr.obj
 0002:000008a4       ??_C@_0BE@ICMCHPHH@Directory?5not?5empty?$AA@ 0040f8a4     LIBCMT:syserr.obj
 0002:000008b8       ??_C@_0BJ@IHEHINLI@Function?5not?5implemented?$AA@ 0040f8b8     LIBCMT:syserr.obj
 0002:000008d4       ??_C@_0BD@CLHBCGPB@No?5locks?5available?$AA@ 0040f8d4     LIBCMT:syserr.obj
 0002:000008e8       ??_C@_0BC@BEDIHIDK@Filename?5too?5long?$AA@ 0040f8e8     LIBCMT:syserr.obj
 0002:000008fc       ??_C@_0BK@JAEBMJJM@Resource?5deadlock?5avoided?$AA@ 0040f8fc     LIBCMT:syserr.obj
 0002:00000918       ??_C@_0BB@FCBJFCAJ@Result?5too?5large?$AA@ 0040f918     LIBCMT:syserr.obj
 0002:0000092c       ??_C@_0N@MMJPGLJK@Domain?5error?$AA@ 0040f92c     LIBCMT:syserr.obj
 0002:0000093c       ??_C@_0M@LHEPIIOM@Broken?5pipe?$AA@ 0040f93c     LIBCMT:syserr.obj
 0002:00000948       ??_C@_0P@PKCJJLLM@Too?5many?5links?$AA@ 0040f948     LIBCMT:syserr.obj
 0002:00000958       ??_C@_0BG@DDBFNKBH@Read?9only?5file?5system?$AA@ 0040f958     LIBCMT:syserr.obj
 0002:00000970       ??_C@_0N@FEHLOILP@Invalid?5seek?$AA@ 0040f970     LIBCMT:syserr.obj
 0002:00000980       ??_C@_0BI@FEALHKLD@No?5space?5left?5on?5device?$AA@ 0040f980     LIBCMT:syserr.obj
 0002:00000998       ??_C@_0P@LFMMIPAE@File?5too?5large?$AA@ 0040f998     LIBCMT:syserr.obj
 0002:000009a8       ??_C@_0CE@ONOKNLPF@Inappropriate?5I?1O?5control?5operat@ 0040f9a8     LIBCMT:syserr.obj
 0002:000009cc       ??_C@_0BE@INBJMKGG@Too?5many?5open?5files?$AA@ 0040f9cc     LIBCMT:syserr.obj
 0002:000009e0       ??_C@_0BO@IIFBODJE@Too?5many?5open?5files?5in?5system?$AA@ 0040f9e0     LIBCMT:syserr.obj
 0002:00000a00       ??_C@_0BB@HMGGCEBG@Invalid?5argument?$AA@ 0040fa00     LIBCMT:syserr.obj
 0002:00000a14       ??_C@_0P@NDHGCGKE@Is?5a?5directory?$AA@ 0040fa14     LIBCMT:syserr.obj
 0002:00000a24       ??_C@_0BA@CJBACOOL@Not?5a?5directory?$AA@ 0040fa24     LIBCMT:syserr.obj
 0002:00000a34       ??_C@_0P@NLEIANHE@No?5such?5device?$AA@ 0040fa34     LIBCMT:syserr.obj
 0002:00000a44       ??_C@_0O@OAMDNOCP@Improper?5link?$AA@ 0040fa44     LIBCMT:syserr.obj
 0002:00000a54       ??_C@_0M@NAAJNNGH@File?5exists?$AA@ 0040fa54     LIBCMT:syserr.obj
 0002:00000a60       ??_C@_0BA@BIBLIOEK@Resource?5device?$AA@ 0040fa60     LIBCMT:syserr.obj
 0002:00000a70       ??_C@_0O@NIPGCINC@Unknown?5error?$AA@ 0040fa70     LIBCMT:syserr.obj
 0002:00000a80       ??_C@_0M@LOEHLCJD@Bad?5address?$AA@ 0040fa80     LIBCMT:syserr.obj
 0002:00000a8c       ??_C@_0BC@HFNFNKAI@Permission?5denied?$AA@ 0040fa8c     LIBCMT:syserr.obj
 0002:00000aa0       ??_C@_0BB@IMDKMPFB@Not?5enough?5space?$AA@ 0040faa0     LIBCMT:syserr.obj
 0002:00000ab4       ??_C@_0CB@EPFKGNAK@Resource?5temporarily?5unavailable@ 0040fab4     LIBCMT:syserr.obj
 0002:00000ad8       ??_C@_0BD@LOHELEP@No?5child?5processes?$AA@ 0040fad8     LIBCMT:syserr.obj
 0002:00000aec       ??_C@_0BE@NFGDDCEF@Bad?5file?5descriptor?$AA@ 0040faec     LIBCMT:syserr.obj
 0002:00000b00       ??_C@_0BC@HKPNECK@Exec?5format?5error?$AA@ 0040fb00     LIBCMT:syserr.obj
 0002:00000b14       ??_C@_0BC@MFFGCDFL@Arg?5list?5too?5long?$AA@ 0040fb14     LIBCMT:syserr.obj
 0002:00000b28       ??_C@_0BK@DPKMCKJ@No?5such?5device?5or?5address?$AA@ 0040fb28     LIBCMT:syserr.obj
 0002:00000b44       ??_C@_0BD@KKNFOBBD@Input?1output?5error?$AA@ 0040fb44     LIBCMT:syserr.obj
 0002:00000b58       ??_C@_0BK@FJBOAFDK@Interrupted?5function?5call?$AA@ 0040fb58     LIBCMT:syserr.obj
 0002:00000b74       ??_C@_0BA@FKIAIBGA@No?5such?5process?$AA@ 0040fb74     LIBCMT:syserr.obj
 0002:00000b84       ??_C@_0BK@FMDHKPNF@No?5such?5file?5or?5directory?$AA@ 0040fb84     LIBCMT:syserr.obj
 0002:00000ba0       ??_C@_0BI@BJFCGOHL@Operation?5not?5permitted?$AA@ 0040fba0     LIBCMT:syserr.obj
 0002:00000bb8       ??_C@_08INEPGKHH@No?5error?$AA@ 0040fbb8     LIBCMT:syserr.obj
 0002:00000bc4       ??_C@_07EPKMNAGK@?4mixcrt?$AA@ 0040fbc4     LIBCMT:tidtable.obj
 0002:00000bcc       ??_C@_0O@NLDKAIKN@EncodePointer?$AA@ 0040fbcc     LIBCMT:tidtable.obj
 0002:00000bdc       ??_C@_0N@NHGLKGEC@KERNEL32?4DLL?$AA@ 0040fbdc     LIBCMT:tidtable.obj
 0002:00000bec       ??_C@_0O@KBPMFGHI@DecodePointer?$AA@ 0040fbec     LIBCMT:tidtable.obj
 0002:00000bfc       ??_C@_07PEJMOBNF@FlsFree?$AA@ 0040fbfc     LIBCMT:tidtable.obj
 0002:00000c04       ??_C@_0M@JCPCPOEF@FlsSetValue?$AA@ 0040fc04     LIBCMT:tidtable.obj
 0002:00000c10       ??_C@_0M@GDNOONDI@FlsGetValue?$AA@ 0040fc10     LIBCMT:tidtable.obj
 0002:00000c1c       ??_C@_08KNHFBNJ@FlsAlloc?$AA@ 0040fc1c     LIBCMT:tidtable.obj
 0002:00000c4c       ??_C@_0CG@PKBDLMEO@InitializeCriticalSectionAndSpin@ 0040fc4c     LIBCMT:initcrit.obj
 0002:00000c74       ??_C@_0N@MDJJJHMB@kernel32?4dll?$AA@ 0040fc74     LIBCMT:initcrit.obj
 0002:00000d08       ??_C@_0BI@DFKBFLJE@GetProcessWindowStation?$AA@ 0040fd08     LIBCMT:crtmbox.obj
 0002:00000d20       ??_C@_0BK@CIDNPOGP@GetUserObjectInformationA?$AA@ 0040fd20     LIBCMT:crtmbox.obj
 0002:00000d3c       ??_C@_0BD@HHGDFDBJ@GetLastActivePopup?$AA@ 0040fd3c     LIBCMT:crtmbox.obj
 0002:00000d50       ??_C@_0BA@HNOPNCHB@GetActiveWindow?$AA@ 0040fd50     LIBCMT:crtmbox.obj
 0002:00000d60       ??_C@_0M@CHKKJDAI@MessageBoxA?$AA@ 0040fd60     LIBCMT:crtmbox.obj
 0002:00000d6c       ??_C@_0L@NDEGIDAG@USER32?4DLL?$AA@ 0040fd6c     LIBCMT:crtmbox.obj
 0002:00000d78       ??_C@_13NOLLCAOD@?$AA?$AA?$AA?$AA@ 0040fd78     LIBCMT:a_map.obj
 0002:00000d80       ___newctype                0040fd80     LIBCMT:ctype.obj
 0002:00001080       __wctype                   00410080     LIBCMT:ctype.obj
 0002:00001288       ___newclmap                00410288     LIBCMT:ctype.obj
 0002:00001408       ___newcumap                00410408     LIBCMT:ctype.obj
 0002:00001588       ??_C@_08JCCMCCIL@HH?3mm?3ss?$AA@ 00410588     LIBCMT:strftime.obj
 0002:00001594       ??_C@_0BE@CKGJFCPC@dddd?0?5MMMM?5dd?0?5yyyy?$AA@ 00410594     LIBCMT:strftime.obj
 0002:000015a8       ??_C@_08BPBNCDIB@MM?1dd?1yy?$AA@ 004105a8     LIBCMT:strftime.obj
 0002:000015b4       ??_C@_02CJNFDJBF@PM?$AA@   004105b4     LIBCMT:strftime.obj
 0002:000015b8       ??_C@_02DEDBPAFC@AM?$AA@   004105b8     LIBCMT:strftime.obj
 0002:000015bc       ??_C@_08EDHMEBNP@December?$AA@ 004105bc     LIBCMT:strftime.obj
 0002:000015c8       ??_C@_08HCHEGEOA@November?$AA@ 004105c8     LIBCMT:strftime.obj
 0002:000015d4       ??_C@_07JJNFCEND@October?$AA@ 004105d4     LIBCMT:strftime.obj
 0002:000015dc       ??_C@_09BHHEALKD@September?$AA@ 004105dc     LIBCMT:strftime.obj
 0002:000015e8       ??_C@_06LBBHFDDG@August?$AA@ 004105e8     LIBCMT:strftime.obj
 0002:000015f0       ??_C@_04MIEPOIFP@July?$AA@ 004105f0     LIBCMT:strftime.obj
 0002:000015f8       ??_C@_04CNLMGBGM@June?$AA@ 004105f8     LIBCMT:strftime.obj
 0002:00001600       ??_C@_05DMJDNLEJ@April?$AA@ 00410600     LIBCMT:strftime.obj
 0002:00001608       ??_C@_05HPCKOFNC@March?$AA@ 00410608     LIBCMT:strftime.obj
 0002:00001610       ??_C@_08GNJGEPFN@February?$AA@ 00410610     LIBCMT:strftime.obj
 0002:0000161c       ??_C@_07CGJPFGJA@January?$AA@ 0041061c     LIBCMT:strftime.obj
 0002:00001624       ??_C@_03MKABNOCG@Dec?$AA@  00410624     LIBCMT:strftime.obj
 0002:00001628       ??_C@_03JPJOFNIA@Nov?$AA@  00410628     LIBCMT:strftime.obj
 0002:0000162c       ??_C@_03BMAOKBAD@Oct?$AA@  0041062c     LIBCMT:strftime.obj
 0002:00001630       ??_C@_03GGCAPAJC@Sep?$AA@  00410630     LIBCMT:strftime.obj
 0002:00001634       ??_C@_03IFJFEIGA@Aug?$AA@  00410634     LIBCMT:strftime.obj
 0002:00001638       ??_C@_03LBGABGKK@Jul?$AA@  00410638     LIBCMT:strftime.obj
 0002:0000163c       ??_C@_03IDFGHECI@Jun?$AA@  0041063c     LIBCMT:strftime.obj
 0002:00001640       ??_C@_03CNMDKL@May?$AA@    00410640     LIBCMT:strftime.obj
 0002:00001644       ??_C@_03LEOLGMJP@Apr?$AA@  00410644     LIBCMT:strftime.obj
 0002:00001648       ??_C@_03ODNJBKGA@Mar?$AA@  00410648     LIBCMT:strftime.obj
 0002:0000164c       ??_C@_03HJBDCHOM@Feb?$AA@  0041064c     LIBCMT:strftime.obj
 0002:00001650       ??_C@_03JIHJHPIE@Jan?$AA@  00410650     LIBCMT:strftime.obj
 0002:00001654       ??_C@_08INBOOONO@Saturday?$AA@ 00410654     LIBCMT:strftime.obj
 0002:00001660       ??_C@_06JECMNKMI@Friday?$AA@ 00410660     LIBCMT:strftime.obj
 0002:00001668       ??_C@_08HACCIKIA@Thursday?$AA@ 00410668     LIBCMT:strftime.obj
 0002:00001674       ??_C@_09DLIGFAKA@Wednesday?$AA@ 00410674     LIBCMT:strftime.obj
 0002:00001680       ??_C@_07BAAGCFCM@Tuesday?$AA@ 00410680     LIBCMT:strftime.obj
 0002:00001688       ??_C@_06JLEDEDGH@Monday?$AA@ 00410688     LIBCMT:strftime.obj
 0002:00001690       ??_C@_06OOPIFAJ@Sunday?$AA@ 00410690     LIBCMT:strftime.obj
 0002:00001698       ??_C@_03FEFJNEK@Sat?$AA@   00410698     LIBCMT:strftime.obj
 0002:0000169c       ??_C@_03IDIOELNC@Fri?$AA@  0041069c     LIBCMT:strftime.obj
 0002:000016a0       ??_C@_03IOFIKPDN@Thu?$AA@  004106a0     LIBCMT:strftime.obj
 0002:000016a4       ??_C@_03MHOMLAJA@Wed?$AA@  004106a4     LIBCMT:strftime.obj
 0002:000016a8       ??_C@_03NAGEINEP@Tue?$AA@  004106a8     LIBCMT:strftime.obj
 0002:000016ac       ??_C@_03PDAGKDH@Mon?$AA@   004106ac     LIBCMT:strftime.obj
 0002:000016b0       ??_C@_03KOEHGMDN@Sun?$AA@  004106b0     LIBCMT:strftime.obj
 0002:000016b4       ??_C@_07GPDNMNG@CONOUT$?$AA@ 004106b4     LIBCMT:initcon.obj
 0002:000016bc       ___dnames                  004106bc     LIBCMT:timeset.obj
 0002:000016d4       ___mnames                  004106d4     LIBCMT:timeset.obj
 0002:00001700       __load_config_used         00410700     LIBCMT:loadcfg.obj
 0002:000017a0       ___safe_se_handler_table   004107a0     <linker-defined>
 0002:000017ac       ___rtc_iaa                 004107ac     LIBCMT:initsect.obj
 0002:000017b0       ___rtc_izz                 004107b0     LIBCMT:initsect.obj
 0002:000017b4       ___rtc_taa                 004107b4     LIBCMT:initsect.obj
 0002:000017b8       ___rtc_tzz                 004107b8     LIBCMT:initsect.obj
 0002:00001c54       __IMPORT_DESCRIPTOR_KERNEL32 00410c54     kernel32:KERNEL32.dll
 0002:00001c68       __NULL_IMPORT_DESCRIPTOR   00410c68     kernel32:KERNEL32.dll
 0003:00000000       __iob                      00412000     LIBCMT:_file.obj
 0003:000003f0       ___app_type                004123f0     LIBCMT:crt0.obj
 0003:000003f4       ___security_cookie         004123f4     LIBCMT:gs_cookie.obj
 0003:000003f8       ___security_cookie_complement 004123f8     LIBCMT:gs_cookie.obj
 0003:00000400       ___badioinfo               00412400     LIBCMT:ioinit.obj
 0003:00000438       __aexit_rtn                00412438     LIBCMT:crt0dat.obj
 0003:00000560       ___nullstring              00412560     LIBCMT:output.obj
 0003:00000564       ___wnullstring             00412564     LIBCMT:output.obj
 0003:00000568       __amblksiz                 00412568     LIBCMT:heapinit.obj
 0003:00000630       __sys_errlist              00412630     LIBCMT:syserr.obj
 0003:000006e0       __sys_nerr                 004126e0     LIBCMT:syserr.obj
 0003:000006e4       ___flsindex                004126e4     LIBCMT:tidtable.obj
 0003:000006e8       ___getvalueindex           004126e8     LIBCMT:tidtable.obj
 0003:000006f0       __lookuptrailbytes         004126f0     LIBCMT:read.obj
 0003:000007f0       __XcptActTab               004127f0     LIBCMT:winxfltr.obj
 0003:00000868       __First_FPE_Indx           00412868     LIBCMT:winxfltr.obj
 0003:0000086c       __Num_FPE                  0041286c     LIBCMT:winxfltr.obj
 0003:00000870       __XcptActTabSize           00412870     LIBCMT:winxfltr.obj
 0003:00000874       __XcptActTabCount          00412874     LIBCMT:winxfltr.obj
 0003:00000878       __cfltcvt_tab              00412878     LIBCMT:cmiscdat.obj
 0003:000008a0       ___initialmbcinfo          004128a0     LIBCMT:mbctype.obj
 0003:00000ac0       __mbctype                  00412ac0     LIBCMT:mbctype.obj
 0003:00000bc8       __mbcasemap                00412bc8     LIBCMT:mbctype.obj
 0003:00000cc8       ___ptmbcinfo               00412cc8     LIBCMT:mbctype.obj
 0003:00000dc4       ___globallocalestatus      00412dc4     LIBCMT:glstatus.obj
 0003:00000dc8       ___clocalestr              00412dc8     LIBCMT:nlsdata2.obj
 0003:00000dd0       ___initiallocinfo          00412dd0     LIBCMT:nlsdata2.obj
 0003:00000ea8       ___ptlocinfo               00412ea8     LIBCMT:nlsdata2.obj
 0003:00000eac       ___lc_clike                00412eac     LIBCMT:nlsdata2.obj
 0003:00000eb0       ___initiallocalestructinfo 00412eb0     LIBCMT:nlsdata2.obj
 0003:00000ed0       __NLG_Destination          00412ed0     LIBCMT:exsup.obj
 0003:00000ee0       ___abort_behavior          00412ee0     LIBCMT:abort.obj
 0003:00000ee4       __pctype                   00412ee4     LIBCMT:ctype.obj
 0003:00000ee8       __pwctype                  00412ee8     LIBCMT:ctype.obj
 0003:00000ef0       ___lc_time_c               00412ef0     LIBCMT:strftime.obj
 0003:00000fa8       ___lc_time_curr            00412fa8     LIBCMT:strftime.obj
 0003:00000fac       ___lconv_static_decimal    00412fac     LIBCMT:lconv.obj
 0003:00000fb0       ___lconv_c                 00412fb0     LIBCMT:lconv.obj
 0003:00000fe0       ___lconv                   00412fe0     LIBCMT:lconv.obj
 0003:00000fe4       ___mb_cur_max              00412fe4     LIBCMT:nlsdata1.obj
 0003:00000fe8       ___decimal_point           00412fe8     LIBCMT:nlsdata1.obj
 0003:00000fec       ___decimal_point_length    00412fec     LIBCMT:nlsdata1.obj
 0003:00000ff0       __coninpfh                 00412ff0     LIBCMT:initcon.obj
 0003:00000ff4       __confh                    00412ff4     LIBCMT:initcon.obj
 0003:00001000       __timezone                 00413000     LIBCMT:timeset.obj
 0003:00001004       __daylight                 00413004     LIBCMT:timeset.obj
 0003:00001008       __dstbias                  00413008     LIBCMT:timeset.obj
 0003:00001090       __tzname                   00413090     LIBCMT:timeset.obj
 0003:000010b0       __lpdays                   004130b0     LIBCMT:days.obj
 0003:000010e4       __days                     004130e4     LIBCMT:days.obj
 0003:00003ca0       __cflush                   00415ca0     LIBCMT:_file.obj
 0003:00003ca8       __aenvptr                  00415ca8     LIBCMT:crt0.obj
 0003:00003cac       __wenvptr                  00415cac     LIBCMT:crt0.obj
 0003:00003cb0       ___error_mode              00415cb0     LIBCMT:crt0.obj
 0003:00003fdc       __maxwait                  00415fdc     LIBCMT:crtheap.obj
 0003:00003fe0       __umaskval                 00415fe0     LIBCMT:crt0dat.obj
 0003:00003fe4       __osplatform               00415fe4     LIBCMT:crt0dat.obj
 0003:00003fe8       __osver                    00415fe8     LIBCMT:crt0dat.obj
 0003:00003fec       __winver                   00415fec     LIBCMT:crt0dat.obj
 0003:00003ff0       __winmajor                 00415ff0     LIBCMT:crt0dat.obj
 0003:00003ff4       __winminor                 00415ff4     LIBCMT:crt0dat.obj
 0003:00003ff8       ___argc                    00415ff8     LIBCMT:crt0dat.obj
 0003:00003ffc       ___argv                    00415ffc     LIBCMT:crt0dat.obj
 0003:00004000       ___wargv                   00416000     LIBCMT:crt0dat.obj
 0003:00004004       __environ                  00416004     LIBCMT:crt0dat.obj
 0003:00004008       ___initenv                 00416008     LIBCMT:crt0dat.obj
 0003:0000400c       __wenviron                 0041600c     LIBCMT:crt0dat.obj
 0003:00004010       ___winitenv                00416010     LIBCMT:crt0dat.obj
 0003:00004014       __pgmptr                   00416014     LIBCMT:crt0dat.obj
 0003:00004018       __wpgmptr                  00416018     LIBCMT:crt0dat.obj
 0003:0000401c       __exitflag                 0041601c     LIBCMT:crt0dat.obj
 0003:00004020       __C_Termination_Done       00416020     LIBCMT:crt0dat.obj
 0003:00004024       __C_Exit_Done              00416024     LIBCMT:crt0dat.obj
 0003:00004178       __stdbuf                   00416178     LIBCMT:_sftbuf.obj
 0003:00004180       ___pInvalidArgHandler      00416180     LIBCMT:invarg.obj
 0003:00004184       __crtheap                  00416184     LIBCMT:heapinit.obj
 0003:00004188       ___sbh_pHeaderDefer        00416188     LIBCMT:sbheap.obj
 0003:000044a4       ?_pnhHeap@@3P6AHI@ZA       004164a4     LIBCMT:handler.obj
 0003:000044a8       __newmode                  004164a8     LIBCMT:_newmode.obj
 0003:000044ac       _gpFlsAlloc                004164ac     LIBCMT:tidtable.obj
 0003:000044b0       _gpFlsGetValue             004164b0     LIBCMT:tidtable.obj
 0003:000044b4       _gpFlsSetValue             004164b4     LIBCMT:tidtable.obj
 0003:000044b8       _gpFlsFree                 004164b8     LIBCMT:tidtable.obj
 0003:000045d0       ?__pInconsistency@@3P6AXXZA 004165d0     LIBCMT:hooks.obj
 0003:000045f4       ___pPurecall               004165f4     LIBCMT:inithelp.obj
 0003:000045fc       ___mbulinfo                004165fc     LIBCMT:mbctype.obj
 0003:00004608       ___mbcodepage              00416608     LIBCMT:mbctype.obj
 0003:0000460c       ___ismbcodepage            0041660c     LIBCMT:mbctype.obj
 0003:00004610       ___mblcid                  00416610     LIBCMT:mbctype.obj
 0003:00004614       ___locale_changed          00416614     LIBCMT:setlocal.obj
 0003:00004618       ___lc_handle               00416618     LIBCMT:nlsdata2.obj
 0003:00004630       ___lc_codepage             00416630     LIBCMT:nlsdata2.obj
 0003:00004634       ___lc_collate_cp           00416634     LIBCMT:nlsdata2.obj
 0003:0000464c       __fmode                    0041664c     LIBCMT:txtmode.obj
 0003:00004650       __commode                  00416650     LIBCMT:ncommode.obj
 0003:0000465c       ___lconv_static_null       0041665c     LIBCMT:lconv.obj
 0003:0000471c       __debugger_hook_dummy      0041671c     <common>
 0003:00004720       ___use_sse2_mathfcns       00416720     <common>
 0003:00004724       ___sse2_available          00416724     <common>
 0003:00004728       ___sbh_cntHeaderList       00416728     <common>
 0003:0000472c       ___sbh_pHeaderList         0041672c     <common>
 0003:00004730       ___sbh_threshold           00416730     <common>
 0003:00004734       ___sbh_pHeaderScan         00416734     <common>
 0003:00004738       ___sbh_sizeHeaderList      00416738     <common>
 0003:0000473c       ___sbh_indGroupDefer       0041673c     <common>
 0003:00004740       ___active_heap             00416740     <common>
 0003:00004744       __pDestructExceptionObject 00416744     <common>
 0003:00004748       ___env_initialized         00416748     <common>
 0003:0000474c       ___onexitend               0041674c     <common>
 0003:00004750       ___onexitbegin             00416750     <common>
 0003:00004754       ___mbctype_initialized     00416754     <common>
 0003:00004758       __FPinit                   00416758     <common>
 0003:0000475c       ___dyn_tls_init_callback   0041675c     <common>
 0003:00004760       __nhandle                  00416760     <common>
 0003:00004780       ___pioinfo                 00416780     <common>
 0003:00004880       __acmdln                   00416880     <common>
 0003:00004884       ___piob                    00416884     <common>
 0003:000048a0       __bufin                    004168a0     <common>
 0003:000058a0       __nstream                  004178a0     <common>

 entry point at        0001:00003dec

 Static symbols

 0001:000005f6       _newstm                    004015f6 f    CIL library: CIL module
 0001:0000078b       _fz_readbyte               0040178b f    CIL library: CIL module
 0001:000007ab       _fz_peekbyte               004017ab f    CIL library: CIL module
 0001:000007c5       _iswhite                   004017c5 f    CIL library: CIL module
 0001:000007e9       _isregular                 004017e9 f    CIL library: CIL module
 0001:00000830       _isnumber                  00401830 f    CIL library: CIL module
 0001:00000850       _fromhex                   00401850 f    CIL library: CIL module
 0001:00000877       _lexname                   00401877 f    CIL library: CIL module
 0001:000008fe       _lexstring                 004018fe f    CIL library: CIL module
 0001:00000a33       _lexhexstring              00401a33 f    CIL library: CIL module
 0001:00000ab6       _pdf_tokenfromkeyword      00401ab6 f    CIL library: CIL module
 0001:0000103a       _addtable                  0040203a f    CIL library: CIL module
 0001:000010b8       _addrange                  004020b8 f    CIL library: CIL module
 0001:000012a7       _cmprange                  004022a7 f    CIL library: CIL module
 0001:0000152e       _pdf_cmaptokenfromkeyword  0040252e f    CIL library: CIL module
 0001:0000176f       _codefromstring            0040276f f    CIL library: CIL module
 0001:0000178c       _lexcmap                   0040278c f    CIL library: CIL module
 0001:000017cf       _parsecmapname             004027cf f    CIL library: CIL module
 0001:0000186a       _parsewmode                0040286a f    CIL library: CIL module
 0001:00001902       _parsecodespacerange       00402902 f    CIL library: CIL module
 0001:00001a69       _parsecidrange             00402a69 f    CIL library: CIL module
 0001:00001c09       _parsecidchar              00402c09 f    CIL library: CIL module
 0001:00001d2c       _parsebfrangearray         00402d2c f    CIL library: CIL module
 0001:00001e4c       _parsebfrange              00402e4c f    CIL library: CIL module
 0001:000020df       _parsebfchar               004030df f    CIL library: CIL module
 0001:00003690       _swap                      00404690 f   LIBCMT:qsort.obj
 0001:000036c0       _shortsort                 004046c0 f   LIBCMT:qsort.obj
 0001:00003bd1       _fast_error_exit           00404bd1 f   LIBCMT:crt0.obj
 0001:00003bf5       _check_managed_app         00404bf5 f   LIBCMT:crt0.obj
 0001:00003c36       ___tmainCRTStartup         00404c36 f   LIBCMT:crt0.obj
 0001:0000431d       __initterm                 0040531d f   LIBCMT:crt0dat.obj
 0001:0000445a       _doexit                    0040545a f   LIBCMT:crt0dat.obj
 0001:0000466c       _flsall                    0040566c f   LIBCMT:fflush.obj
 0001:00004a3d       _write_char                00405a3d f   LIBCMT:output.obj
 0001:00004a70       _write_multi_char          00405a70 f   LIBCMT:output.obj
 0001:00004a94       _write_string              00405a94 f   LIBCMT:output.obj
 0001:00006a7e       __use_encode_pointer       00407a7e f   LIBCMT:tidtable.obj
 0001:000070ed       _fastcopy_I                004080ed f   LIBCMT:p4_memcpy.obj
 0001:000089ae       ?strtoxl@@YAKPAUlocaleinfo_struct@@PBDPAPBDHH@Z 004099ae f   LIBCMT:strtol.obj
 0001:00009064       __unwind_handler4          0040a064 f   LIBCMT:exsup4.obj
 0001:000093ac       _parse_cmdline             0040a3ac f   LIBCMT:stdargv.obj
 0001:00009820       ___crtInitCritSecNoSpinCount@8 0040a820 f   LIBCMT:initcrit.obj
 0001:00009b01       __onexit_nolock            0040ab01 f   LIBCMT:onexit.obj
 0001:00009dfe       _siglookup                 0040adfe f   LIBCMT:winsig.obj
 0001:0000a142       ?CPtoLCID@@YAHH@Z          0040b142 f   LIBCMT:mbctype.obj
 0001:0000a171       ?setSBCS@@YAXPAUthreadmbcinfostruct@@@Z 0040b171 f   LIBCMT:mbctype.obj
 0001:0000a1c6       ?setSBUpLow@@YAXPAUthreadmbcinfostruct@@@Z 0040b1c6 f   LIBCMT:mbctype.obj
 0001:0000a3f4       ?getSystemCP@@YAHH@Z       0040b3f4 f   LIBCMT:mbctype.obj
 0001:0000aa51       __updatetlocinfoEx_nolock  0040ba51 f   LIBCMT:setlocal.obj
 0001:0000b1c9       _fastzero_I                0040c1c9 f   LIBCMT:p4_memset.obj
 0001:0000b338       _has_osfxsr_set            0040c338 f   LIBCMT:cpu_disp.obj
 0001:0000b6d4       __tsopen_nolock            0040c6d4 f   LIBCMT:open.obj
 0001:0000c39c       __unwind_handler           0040d39c f   LIBCMT:exsup.obj
 0001:0000c4b3       ?x_ismbbtype_l@@YAHPAUlocaleinfo_struct@@IHH@Z 0040d4b3 f   LIBCMT:ismbbyte.obj
 0001:0000c65a       ?__crtLCMapStringA_stat@@YAHPAUlocaleinfo_struct@@KKPBDHPADHHH@Z 0040d65a f   LIBCMT:a_map.obj
 0001:0000ca3f       ?__crtGetStringTypeA_stat@@YAHPAUlocaleinfo_struct@@KPBDHPAGHHH@Z 0040da3f f   LIBCMT:a_str.obj
